:1000000009C00EC00DC00CC00BC00AC009C008C09A
:1000100007C006C011241FBECFE9CDBF58D09AC07B
:10002000EFCF8FE187BB80E288BB089583E090E04B
:10003000C3982FE339E141E0215030404040E1F7DF
:1000400000C00000C39A2FE339E141E02150304065
:100050004040E1F700C00000C3980197009741F7C6
:10006000089583E090E0C2982FE339E141E0215008
:1000700030404040E1F700C00000C29A2FE339E170
:1000800041E0215030404040E1F700C00000C298FC
:100090000197009741F708958AE090E022E028BB9D
:1000A0003FE349E151E0315040405040E1F700C0AA
:1000B000000018BA3FE349E151E031504040504060
:1000C000E1F700C000000197009749F70895A9DF04
:1000D000C1E0D0E0CC24C394D12C0F2EF9E0EF2E58
:1000E000F02D0F2EF3E0FF2EF02D04E112E12BC0D6
:1000F000E8BA2FE78FE492E1215080409040E1F789
:1001000000C0000093DFF8BA2FE789EA93E021509E
:1001100080409040E1F700C0000008BB2FE78FE46B
:1001200092E1215080409040E1F700C0000099DF4B
:1001300018BB2FE789EA93E0215080409040E1F717
:1001400000C000002196C630D10594F2A5DFCC2D69
:08015000DD2DF9CFF894FFCF7B
:00000001FF
